:100000000C9461010C9489010C9489010C94890170
:100010000C9489010C9489010C9489010C94890138
:100020000C9489010C9489010C9481060C944D0563
:100030000C9489010C9489010C9489010C94890118
:100040000C9489010C9489010C9489010C94890108
:100050000C9489010C9489010C9489010C94BA01C7
:100060000C9489010C9489010C9489010C948901E8
:100070000C9489010C9489010C9489010C948901D8
:100080000C9489010C9489010C9489010C948901C8
:100090000C9489010C9489010C9489010C948901B8
:1000A0000C9489010C9489010C948901BD02C00251
:1000B000AF02B302B902E102E102E102C402C802E6
:1000C000CC02D202D602E102DC02000000020009EA
:1000D0000F0000030401000C0000000000000000FD
:1000E00000000000000000000408020110408040F1
:1000F000102040804080080204018040201002014E
:10010000108010204040040404040403040502028B
:1001100002020403020202020606060606060404A0
:100120000202020400000000250028002B002E001F
:10013000310000000000240027002A002D003000BC
:1001400000C18081C11201000202000040EB0304E3
:10015000240001010200011201000200000040EB36
:1001600003042400010102000152424C00426C656C
:100170006E64204D6963726F0004030904080B006C
:10018000020202010009040000010202000005242D
:1001900000100105240101010424020605240600C3
:1001A000010705810310004009040100020A000054
:1001B000000705020240000007058302400000001E
:1001C000000000000000002A2B28000000000000B2
:1001D0000000000000000000000000000000002CF3
:1001E0009EB4A0A1A2A434A6A7A5AE362D37382769
:1001F0001E1F20212223242526B333B62EB7B89FF5
:100200008485868788898A8B8C8D8E8F9091929336
:100210009495969798999A9B9C9D2F3130A3AD35D4
:100220000405060708090A0B0C0D0E0F1011121316
:100230001415161718191A1B1C1DAFB1B0B50009FB
:1002400004020001030000000921010100012265F0
:10025000000705840340000105010902A10109010D
:10026000A100850105091901290315002501950340
:100270007501810295017505810305010930093178
:1002800009381581257F750895038106C0C00501D1
:100290000906A1018502050719E029E715002501D6
:1002A0007501950881029501750881039506750809
:1002B000150025650507190029658100C000B507EF
:1002C000080911241FBECFEFDAE0DEBFCDBF11E079
:1002D000A0E0B1E0EAE8F2E102C005900D92A83298
:1002E000B107D9F721E0A8E2B1E001C01D92A7391A
:1002F000B207E1F712E0C2ECD2E004C02297FE019F
:100300000E943F09CE3BD107C9F70E94A3010C947C
:1003100043090C94000061E08DE00C94E20261E07E
:100320008DE00E941B0368EE73E080E090E00E9485
:10033000270260E08DE00E941B0368EE73E080E01E
:1003400090E00C9427020E944F0281E391E00E940A
:10035000D70689B5806189BD09B400FEFDCF0E9432
:100360008B01C0E0D0E00E948F012097E1F30E9452
:100370000000F9CF1F920F920FB60F9211242F9306
:100380003F938F939F93AF93BF9380912901909157
:100390002A01A0912B01B0912C013091280126E077
:1003A000230F2D3720F40296A11DB11D05C029E8A9
:1003B000230F0396A11DB11D2093280180932901CD
:1003C00090932A01A0932B01B0932C0180912D01D1
:1003D00090912E01A0912F01B09130010196A11DA5
:1003E000B11D80932D0190932E01A0932F01B09306
:1003F0003001BF91AF919F918F913F912F910F90BD
:100400000FBE0F901F9018953FB7F89480912D0163
:1004100090912E01A0912F01B091300126B5A89B9B
:1004200005C02F3F19F00196A11DB11D3FBF6627E2
:10043000782F892F9A2F620F711D811D911D43E026
:10044000660F771F881F991F4A95D1F70895CF929D
:10045000DF92EF92FF92CF93DF936B017C010E94BA
:100460000402EB01C114D104E104F10489F00E94FB
:10047000F7060E9404026C1B7D0B683E734090F3EC
:1004800081E0C81AD108E108F108C851DC4FEACF71
:10049000DF91CF91FF90EF90DF90CF900895789407
:1004A00084B5826084BD84B5816084BD85B5826079
:1004B00085BD85B5816085BDEEE6F0E08081816017
:1004C0008083E1E8F0E01082808182608083808117
:1004D00081608083E0E8F0E0808181608083E1E9F1
:1004E000F0E0808182608083808181608083E0E9A8
:1004F000F0E0808181608083E1ECF0E080818460C5
:100500008083808182608083808181608083E3EC4E
:10051000F0E0808181608083E0ECF0E080818260A7
:100520008083E2ECF0E0808181608083EAE7F0E0A4
:1005300080818460808380818260808380818E7FDF
:100540008083808180688083089590E0FC013197EA
:10055000EF30F105B0F5EA5AFF4F0C943D09809158
:1005600080008F7703C0809180008F7D8093800012
:10057000089580918000877FF9CF84B58F7702C07E
:1005800084B58F7D84BD0895809190008F7707C0DA
:10059000809190008F7D03C080919000877F809331
:1005A000900008958091C0008F7703C08091C000B3
:1005B0008F7D8093C00008958091C200877F8093D3
:1005C000C2000895CF93DF9390E0FC01E851FF4F04
:1005D0002491FC01EA5FFE4F8491882349F190E069
:1005E000880F991FFC01EE5CFE4FA591B4918C5DC4
:1005F0009E4FFC01C591D4919FB7611108C0F8943A
:100600008C91209582238C93888182230AC062304A
:1006100051F4F8948C91322F309583238C938881F8
:10062000822B888304C0F8948C91822B8C939FBF7B
:10063000DF91CF9108950F931F93CF93DF931F9274
:10064000CDB7DEB7282F30E0F901E653FF4F849194
:10065000F901E851FF4F1491F901EA5FFE4F04914F
:100660000023C9F0882321F069830E94A5026981D3
:10067000E02FF0E0EE0FFF1FEC5DFE4FA591B4916F
:100680009FB7F8948C91611103C01095812301C02C
:10069000812B8C939FBF0F90DF91CF911F910F9172
:1006A00008954091350150913601209133013091E8
:1006B000340142175307B4F49091E8009570E1F3C8
:1006C0009091E80092FD19C08093F100809135016E
:1006D0009091360101968F739927892B19F48EEF2B
:1006E0008093E800809135019091360101969093B6
:1006F00036018093350181E0089580E00895CF921E
:10070000DF92FF920F931F93CF93DF931F92CDB78A
:10071000DEB7082F162F862F880F8E5F99830E94D1
:10072000510383E00E945103F02EC02E9981D92EEF
:100730008C2D8F19811778F4F60184910E94510352
:10074000082F80E00E9451038023FFEFCF1ADF0AB9
:100750008111EECF01C081E00F90DF91CF911F9109
:100760000F91FF90DF90CF900895615030F020916D
:10077000F100FC0120830196F8CF289A84E680934B
:10078000380108952FB7FC012083F89467706093B7
:10079000E9000895CF93DF931F92CDB7DEB7682F9E
:1007A000CE0101960E94C2038091F20099819FBF01
:1007B0000F90DF91CF910895FF920F931F93CF93E6
:1007C000DF9300D0CDB7DEB7F62E8A0190913701C6
:1007D000992311F057FF03C08FEF9FEF2BC0682FB5
:1007E000CE0101967A830E94C2038091F20090E0CC
:1007F000A8017A81801791070CF4AC01EF2DF72F37
:10080000F40E84E6FE1639F0289A80933801909110
:10081000F1009193F7CF4115510521F08091F2003D
:10082000882321F089818FBFCA0104C08BE68093A1
:10083000E800F8CF0F900F90DF91CF911F910F91AB
:10084000FF900895CF93DF931F92CDB7DEB741E0BD
:1008500050E0BE016F5F7F4F0E94DC03019719F4E7
:10086000898190E002C08FEF9FEF0F90DF91CF91D1
:100870000895CF93DF931F92CDB7DEB7682FCE01D7
:1008800001960E94C2039091E800892F807295FF23
:1008900004C09091F20080E4891B99819FBF0F9062
:1008A000DF91CF9108956F927F928F929F92AF9236
:1008B000BF92CF92DF92EF92FF920F931F93CF934D
:1008C000DF931F92CDB7DEB7782E7B01C42EB52EF5
:1008D00080913701882369F0042F152F8AEFD82ED5
:1008E000872D8072982E9AE3A92E872D8074882EEA
:1008F00011C08FEF9FEF57C0872D0E943904682EDB
:1009000081110CC0DA94A9F361E070E080E090E01E
:100910000E9427020115110579F73BC0282F30E00E
:10092000021713070CF4602E672DCE0101960E946A
:10093000C2038091E80085FF29C0262D30E0021B0C
:10094000130B992039F06A948FEF6816B1F010926A
:10095000F100F9CFF701862D77FE07C0815058F0DE
:1009600094919093F1003196F9CF815020F09191BC
:100970009093F100FACFE20EF31E8091E80085FF1C
:100980000FC00115110511F481100AC089818FBFB4
:10099000C1CF5D9A84E6809339018C2D9B2D03C0D5
:1009A000A092E800F3CF0F90DF91CF911F910F91AC
:1009B000FF90EF90DF90CF90BF90AF909F908F907F
:1009C0007F906F9008951092E90010923601109276
:1009D000350190933401809333010895CF92DF92D3
:1009E000FF920F931F93CF93DF9300D0CDB7DEB765
:1009F000F82E8A016B0101151105B1F0F601F7FE21
:100A000002C0849101C0808149835A830E945103AE
:100A100001501109FFEFCF1ADF0A49815A81811174
:100A2000EACF8FEF9FEF01C0CA010F900F90DF91C7
:100A3000CF911F910F91FF90DF90CF9008951F935A
:100A4000CF93DF931F92CDB7DEB7162F2091E8002A
:100A500022FFFCCF612F79830E94B5038BEF809337
:100A6000E800812F7981972F0F90DF91CF911F910F
:100A70000895CF93DF931F92CDB7DEB71982CE01D1
:100A800001960E945507CE0101960E94F0078981C8
:100A900090E00F90DF91CF9108951F920F920FB6C3
:100AA0000F921124EF92FF920F931F932F933F9376
:100AB0004F935F936F937F938F939F93AF93BF9366
:100AC000EF93FF93CF93DF93CDB7DEB76297DEBF8F
:100AD000CDBF1092E9008091E80083FFEBC068E091
:100AE000CE010A960E94B50382EF8093E8009A85B2
:100AF00097FF05C08091E80080FFFCCF03C08EEF18
:100B00008093E800892F807609F0B9C08B85811128
:100B100005C01092F1001092F100C5C0282F2D7F62
:100B2000213009F4C0C0853049F48091E80080FF8D
:100B3000FCCF8C8580688093E300B5C0863009F0D7
:100B400076C02D85E888F988223071F580E090E044
:100B50002A8B0E94E3040E94390599E08E010F5F01
:100B60001F4FF801392F11923A95E9F799832A8995
:100B70002A8391E09E8390E898879AEF9987209145
:100B8000350130913601275F3F4F3C832B838D83A6
:100B9000C7010E94E30449E050E0B80180E00E94F0
:100BA000EE040E9439057FC0C7012A8B0E94E3042E
:100BB0002A89223241F482E290E00E94FB07892BCD
:100BC00009F071C074C0213069F488899989089747
:100BD00011F42093320180913201811118C067E530
:100BE00071E01AC0233009F062C08C85882391F02F
:100BF000823021F46BE08DE691E006C0813009F08F
:100C000056C063E089E691E00E947F034AC065E434
:100C100071E002C069E771E06115710509F447C030
:100C2000FB01449150E080E80E94EE043CC0873014
:100C300009F43DC0883021F481E08093F10033C095
:100C4000893089F5937099F5E1E4F1E081E021E0E4
:100C500096E38093E9002093EB0034913093EC000D
:100C60009093ED008F5F3196853099F78EE78093F2
:100C7000EA001092EA008C858093370114C08889BD
:100C800099890E94E3048E85811105C0CE010A96E0
:100C90000E94600706C0823051F4CE010A960E947D
:100CA0002308882321F08EEF8093E80003C081E2BF
:100CB0008093EB0062960FB6F894DEBF0FBECDBFF7
:100CC000DF91CF91FF91EF91BF91AF919F918F9164
:100CD0007F916F915F914F913F912F911F910F9154
:100CE000FF90EF900F900FBE0F901F90189580937C
:100CF000E9008091F200882319F08AE38093E800EC
:100D000008951F920F920FB60F9211242F933F93C5
:100D10004F935F936F937F938F939F93AF93BF9303
:100D2000EF93FF938091E1001092E10083FF0FC0E9
:100D30001092E90091E09093EB001092EC0092E3A6
:100D40009093ED001092370198E09093F00082FFAD
:100D50001DC083E00E94770680913901882339F015
:100D600080913901815080933901882369F0809105
:100D70003801882359F080913801815080933801DF
:100D8000811104C0289802C05D98F1CFFF91EF91C6
:100D9000BF91AF919F918F917F916F915F914F9193
:100DA0003F912F910F900FBE0F901F9018951092AA
:100DB000370181E08093D70080EA8093D80082E0F9
:100DC00089BD09B400FEFDCF61E070E080E090E0F5
:100DD0000E94270280E98093D8008CE08093E20093
:100DE0001092E000559A209A5D98289808950895E9
:100DF000CF93DF931F92CDB7DEB76983DC01ED910E
:100E0000FC910280F381E02D41E050E0BE016F5F74
:100E10007F4F09950F90DF91CF910895CF93DF9386
:100E2000EC018C859D8597FF05C082E00E9422041D
:100E30009D878C878C859D85DF91CF91089583E078
:100E40000C947706FC018485958597FD06C082E0A9
:100E50000E94CA0390E00196089582E00E94CA03AE
:100E600090E00895FC018485958597FD05C02FEFDE
:100E70003FEF35872487089582E00C942204CF93B6
:100E8000DF93EC0180910701882331F083E00E9419
:100E900053041816190634F081E090E09B838A838E
:100EA00080E090E0DF91CF910895FC0120812E5FDA
:100EB000208342E450E06DE771E080E80C94EE049A
:100EC000FC0181819081913A59F4813209F03CC052
:100ED00047E050E060E071E080E00E94EE0443C033
:100EE000913291F5803239F467E070E080E091E072
:100EF0000E941F0506C0823209F035C082818093AE
:100F000007018091000190910101A0910201B0912F
:100F10000301803B9440A105B105C1F48091070114
:100F200080FD14C087E797E790930108809300083D
:100F30002BE088E190E00FB6F894A89580936000CC
:100F40000FBE209360000FC080E0089588E10FB6C7
:100F5000F89480936000109260000FBEA8951092E4
:100F600001081092000881E0089510923D0110924E
:100F70003C0188EE93E0A0E0B0E080933E019093C6
:100F80003F01A0934001B09341018EE091E0909326
:100F90003B0180933A018FEF9FEF9093470180933D
:100FA00046010895FF920F931F93CF93DF93EC01B7
:100FB000F62EE881F9810480F581E02D09958C01F8
:100FC000E881F9810680F781E02D6F2DCE0109952A
:100FD000C8019927DF91CF911F910F91FF9008953C
:100FE000FC0120812F5F208349E150E06FE372E034
:100FF00080E80C94EE0445E650E068E572E080E895
:101000000C94EE04EF92FF920F931F93CF93DF9314
:101010001F92CDB7DEB789838B017A0141E050E0A2
:10102000BE016F5F7F4F84E00E945304A701B801A7
:1010300084E40E9453040F90DF91CF911F910F9190
:10104000FF90EF900895FC0191818081813A31F405
:1010500081E0913091F0933089F411C0813271F4C4
:101060009B3021F482818093090105C09A3031F4CC
:1010700082818093080181E00895089580E00895B9
:1010800048E050E082E00C940208CF93DF93DC014B
:10109000683818F0E8E7E60F25C0E62FF0E067FFB4
:1010A00011C0E058F10981E090E001C0880FEA9595
:1010B000EAF714969C911497982B14969C93149786
:1010C000E0E010C0E154FE4FE491EE2309F440C08B
:1010D000E7FF08C014968C911497826014968C9345
:1010E0001497EF7716968C9116978E1741F11796F5
:1010F0008C9117978E1719F118968C9118978E1757
:10110000F1F019968C9119978E17C9F01A968C9157
:101110001A978E17A1F01B968C911B978E1779F05A
:1011200080E090E0ED01C80FD91F2E81211102C08F
:10113000EE8305C0019686309105A1F709C0BD0177
:101140006C5F7F4FCD010E94400881E090E008C0B5
:1011500081E090E013969C938E93129780E090E04C
:10116000DF91CF910895683818F0E8E7E60F25C0C1
:10117000E62FF0E067FF12C0E058F10921E030E00F
:1011800001C0220FEA95EAF72095DC0114963C9104
:101190001497322314963C93E0E00FC0E154FE4FC5
:1011A000E491EE2329F1E7FF08C0DC0114962C91AD
:1011B00014972D7F14962C93EF7720E030E0EE23E8
:1011C00051F0DC01A20FB31F16964C9116974E13E7
:1011D00002C016961C922F5F3F4F2630310579F7DB
:1011E000BC016C5F7F4F0E94400881E090E0089551
:1011F00080E090E00895FC01168217821086118627
:10120000128613861482BC016C5F7F4F0C944008D9
:101210001092960110928D0110928C018EE191E056
:1012200090938B0180938A010895CF92DF92EF9281
:10123000FF920F931F93CF93DF936C017A01EB0121
:10124000E60EF71E00E010E0CE15DF0561F06991B3
:10125000D601ED91FC910190F081E02DC601099538
:10126000080F191FF1CFC801DF91CF911F910F9186
:10127000FF90EF90DF90CF900895EE0FFF1F059045
:0A128000F491E02D0994F894FFCFDB
:10128A0000E1000000000000010100000000F80673
:10129A003F07220732070E071F0700000000D20788
:0812AA0015094508B308FB0813
:00000001FF
